:020000020000FC
:0200000007C334
:0200040018954D
:02000800189549
:02000C00189545
:02001000189541
:02001C00189535
:0200240018952D
:020028008BC08B
:02002C00A9C069
:02003000189521
:02004000189511
:0200440062C098
:02004800189509
:02004C00189505
:02005000189501
:020054001895FD
:020058001895F9
:02005C001895F5
:020060001895F1
:020064001895ED
:020068001895E9
:02006C001FC0B3
:020070001895E1
:020074001895DD
:020078001895D9
:02007C001895D5
:020080001895D1
:020084001895CD
:020088001895C9
:02008C001895C5
:020090001895C1
:020094001895BD
:020098001895B9
:02009C001895B5
:0200A0001895B1
:0200A4001895AD
:0200A8001895A9
:1000AC002FB6DF2DCE2DF49BD6300000F499D7302F
:1000BC0039F418607091C9007F7B7093C9001DC022
:1000CC000E947B0E7991FD2EEC2EF09914C0D091EC
:1000DC002F01D03881F00F921F92D79F17FE02C0CC
:1000EC007FEF05C0712D703810F07FEF02C0000C4F
:1000FC00771F1F900F907093CE002FBE18952FB6C0
:10010C000260DD2009F0DA94CA9409F012C07AE09A
:10011C00C72E0460F09B08C000002E9B03C02E98D5
:10012C005D9802C02E9A5D9ABA9409F002C0B72E5F
:10013C000160E3CF2FB67091E10073FF19C070918D
:10014C00E100777E7093E10077277093E90070915E
:10015C00EB0071607093EB0070E07093EC0070E05A
:10016C0072607093ED007091F00078607093F00005
:10017C002FBE18952FB68F937091F40070FF07C0A7
:10018C0070E07093E9007091E80073FD0DD07091F0
:10019C00F40072FDD6D1F79B04C07091F40073FD8E
:1001AC0013D28F912FBE1895EF93FF937091F1009E
:1001BC00709305017091F100709306017091F1003C
:1001CC00709308017091F100709309017091F10026
:1001DC0070930A017091F10070930B017091F10012
:1001EC0070930C017091F10070930D017091E80007
:1001FC00777F7093E80070910501F79B06C0713210
:10020C0009F47DC0713A09F470C0717619F071303F
:10021C0009F00BC070910601703041F07530A9F0F7
:10022C00763039F1793009F485C0E0C077277093C6
:10023C00F1007093F1007091E8007E7F7093E800FC
:10024C007091E80072FFFCCFD6C0709108017F77E7
:10025C007093E3007091E8007E7F7093E8007091DA
:10026C00E80070FFFCCF7091E30070687093E300BE
:10027C00C2C070910901713029F0723069F073308D
:10028C0021F1B4C0F79B03C0EEEFFCE102C0ECEC33
:10029C00FDE1D491B3D0AFC0D0910C01D03049F076
:1002AC0070910D01703029F4F79BD536F799D33442
:1002BC0020F0F79BD5E6F799D3E4F79B03C0E0E574
:1002CC00FDE111C0EAEDFDE10EC07091080177234C
:1002DC0019F4E4E9FDE106C0713019F4E6EAFDE138
:1002EC0001C084C0D491F6D086C0709106017132E1
:1002FC0009F07CC0E2ECFDE1D7E0ECD07CC0709161
:10030C000601703251F47091E80072FFFCCF7091CD
:10031C00E8007B7F7093E80003C0723209F066C07E
:10032C007091E8007E7F7093E8007091E80070FF98
:10033C00FCCF61C0F79BC2E0F799C3E0C093E90022
:10034C007091EB007E7F7093EB007091ED007D7FE0
:10035C007093ED00CA9591F771E07093E90070917C
:10036C00EB0071607093EB0071E87093EC0070E33C
:10037C0072607093ED0077277093F00072E07093C9
:10038C00E9007091EB0071607093EB0070E8709372
:10039C00EC0070E372607093ED007091F000746487
:1003AC007093F000F79B14C073E07093E9007091A8
:1003BC00EB0071607093EB0071EC7093EC0070E1EA
:1003CC0072607093ED007091F00071607093F000AA
:1003DC0077277093E9007091E8007E7F7093E800B6
:1003EC007091E8007170E1F3F69A05C07091EB0022
:1003FC0070627093EB00FF91EF91089570910D0175
:10040C00772331F470910C017D1708F4D72FCC278A
:10041C007091E80072FD94C075917093F100DA95BB
:10042C00C395C830A9F77091E8007E7F7093E800FF
:10043C007091E8007570E1F37091E80072FD80C076
:10044C00EF93FF938F939F935F935527F1E0E8E031
:10045C000E94430B802D0E94430B902D813411F48C
:10046C00933211F0982B41F481E48093F10083E2F4
:10047C008093F1005FEF04C08093F1000092F100D3
:10048C000E94430B802D0E94430B902D873321F447
:10049C00903011F4552321F40E94430B002061F499
:1004AC0087E390E0F79B92E80000F79B86E380934C
:1004BC00F1009093F10006C0F79B01968093F10038
:1004CC009093F1005F919F918F91FF91EF91CCE010
:1004DC00D45014C070910D01772329F470910C0144
:1004EC007D1708F4D72FCC277091E80072FD28C037
:1004FC00A89575917093F100DA95C39577E07C23FC
:10050C0049F47091E8007E7F7093E8007091E800E8
:10051C007570E1F3D03041F77091E800747009F018
:10052C000AC07091E8007E7F7093E800A8957091E6
:10053C00E80072FFFBCF7091E8007B7F7093E800BE
:10054C0008955F9372E07093E9007091E80072FF78
:10055C0039C07091E8007B7F7093E80010FD32C0C9
:10056C007091F200772309F1D62DC72D5091F1002F
:10057C005993D53011F4D2E0C0E06D2E7C2E6F93E0
:10058C00572D662D681430F009F005C0791410F061
:10059C0049F001C06D5F59196809623018F05F3B72
:1005AC0008F011606F917A9509F710FD0BC07091EE
:1005BC00E8007B7F7093E80000007091E8007F7783
:1005CC007093E8005F9108955F9373E07093E90076
:1005DC007091E80070FF14C0707A7093E80011FFFE
:1005EC0009C0C0ECD1E070910F0159915093F1000A
:1005FC007A95D9F71D7F7091E8007F777093E800AA
:10060C005F910895F89491E09EBF9CEF9DBF882761
:10061C009FEF84B995B987B998B98AB99BB98DB947
:10062C009EB980BB91BB002711272227CC24C394F1
:10063C00BC2CF1E0E0E099279193F130E8F3539A68
:10064C005B9A379907C0F1E0E8E055270E944E0B02
:10065C00ED30D9F7519A59980E94C80C992790936C
:10066C0080009CE09093810092E081E79093890058
:10067C008093880092E090936F0090B7906890BF41
:10068C008EE19EE0809360009093600099279EBB62
:10069C000E94370B90931B010E947A0B0E945D0BFA
:1006AC00A895F69BFDCF0E94650B0E94370B90938B
:1006BC001B01559A209A2898269A2E9A5D9AF1E059
:1006CC00E4E00E94430B00922301A895A8954427CF
:1006DC00332718600E94C80C0E941C0C0E943F0A11
:1006EC000E943D0EF49B07C012D7F6F79A35E1F73E
:1006FC00DBD11F78F9CF0BD7F6F7F3D0FCCF6F9384
:10070C008F939F93982F60911101639560931101C2
:10071C0097FF50C0903F29F42160217F90931201E4
:10072C00DCC0973F19F56130A9F1623081F097E098
:10073C0090931001909113019093120190911401D8
:10074C009093130197EF90931401207F95C096E03E
:10075C0090931001909113019093120197EF909345
:10076C001301992790931401207F86C09093120156
:10077C00943FE8F0983F89F09E3F79F09A3F69F0FA
:10078C009B3F59F09C3F49F09F3F39F0963F29F031
:10079C00247F9FC097EF9093120199279093130198
:1007AC009093140195E090931001207F65C0216017
:1007BC00217F93C020FD0CC0207F909312019FE0FD
:1007CC00909310019927909313019093140154C0A6
:1007DC0021FD1EC0909313019927909314019091C1
:1007EC001201913F79F0933F69F0907F903C21F09A
:1007FC00903D11F0226071C0929590931001216090
:10080C00217F3AC092E0909310012160217F34C087
:10081C0020FF5FC022FD18C09093140123FF02C07B
:10082C0024605BC090911201923F49F0903FF9F027
:10083C0092959F70909310012160217F1DC093E0D1
:10084C0090931001207F18C020FF43C022FF41C0AD
:10085C0080911301809312018091140180931301F4
:10086C009093140194E090931001297F05C094E0BB
:10087C0090931001297F2860F894000091E09093E8
:10088C00E900A8959091E80090FFFBCF9E7B909398
:10089C00E800909110019093F100909112019093C7
:1008AC00F100909113019093F100909114019093A9
:1008BC00F1009091E8009E7F9093E80000009091E9
:1008CC00E8009F779093E800789499279093110112
:1008DC0004C0992790931101207F9F918F916F9164
:1008EC000895F09B05C0A8959A3509F0089584C029
:1008FC009A3519F4D9D01F789EC0F0999CC09635C2
:10090C0011F4F8D198C0933511F4DED194C094351C
:10091C0008F064C0903408F026C0933219F40E9499
:10092C00710689C0943219F40E944A3F84C09632F1
:10093C0019F40E94483F7FC09B3219F40E94BA0BF5
:10094C007AC09C3211F4D0D176C09D3219F40E9439
:10095C00CF0B71C09D3311F4D5D16DC09F3319F4F9
:10096C000E94B10868C0903419F40E94180C63C03E
:10097C00913411F458D25FC0923411F40DD25BC093
:10098C00933419F40E94FF0556C0943419F40E9454
:10099C00940C51C0973419F40E940C074CC0983435
:1009AC0019F40E94BE0647C09D3411F4FED143C019
:1009BC009E3439F490913B01923010F00E9439072B
:1009CC003AC0903511F445D236C0913519F40E94D5
:1009DC00860731C0923511F469D22DC0943511F4CB
:1009EC006BD329C0973519F40E94C70624C09835DB
:1009FC0019F40E946C3F1FC0953511F4B8D01BC080
:100A0C009E3519F40E944C3F16C09F3519F40E9474
:100A1C005F3F11C09C3719F40E94B30C0CC09E3779
:100A2C0019F40E94DB0B07C09D3009F435C09A30D5
:100A3C0011F0903209F40895F79909C080912301BF
:100A4C00806C0E9485038FE30E94850305C08FE3B1
:100A5C000E94EA0A0E94E90A2AD692E0692E892E9F
:100A6C0090E0792E992EF8940000E2E0E093E900F2
:100A7C00E091E800EB7FE093E8000000E091E800F3
:100A8C00EF77E093E8001E78F098077E91E09EBF28
:100A9C009CEF9DBF789426CEF49908950000F79BA7
:100AAC0008950E94E90A08959AE0D92EA8952FD5A9
:100ABC00DD2019F4F09BC0CF0895CEF79A35A1F341
:100ACC001F79913A81F01064923A69F09AE0D92E2C
:100ADC00A895DD2039F01BD5E6F79A3529F3953A20
:100AEC0009F0F7CF27C008601061F09AAA27A093ED
:100AFC003B01A0933C01A0933E01BB27F7E0E0E053
:100B0C0096E0D92EDD20B1F002D5E6F7F93008F4E5
:100B1C0091931196BB23A1F3B23011F015FDF0CFD8
:100B2C00A13071F716FF04C015FD02C01062E8CFAA
:100B3C00953A41F08AE548D581EC46D585EA44D50D
:100B4C00077F0895F7E0E0E0B5E0A0E091919D9378
:100B5C00F49903C0B630D1F702C0B730B9F78AE5C3
:100B6C0033D581EC31D585EA2FD5077F08953F9297
:100B7C005F936F930F930062F198F2989FE782EE68
:100B8C000E942C0B98D066F4332E832FF19A3CD50F
:100B9C00F19891D02EF4832FF19A36D5F19801C0AB
:100BAC0026C0532F9FE788EE0E942C0B84D06EF446
:100BBC00832FF19A0E940A0BF198432E7CD02EF4CD
:100BCC00832FF19A21D5F19801C011C0F1E0E8E032
:100BDC005FD5532D5DD5532F5BD5542D59D55AE583
:100BEC0057D5B9D20F916F915F913F9008950C94A6
:100BFC0022059FE78AEC2AD58AE3E6D482E004D367
:100C0C000EF03BC00F7E3A3010F4832F04C081E30A
:100C1C00DBD4832F8A50805D0E94EA0A532F552320
:100C2C0061F1513150F55F939FE788ED0FD59FE748
:100C3C008AEC0CD58AE3C8D482E0E6D25F910EF040
:100C4C001CC00F7E3A3010F4832F04C081E3BCD457
:100C5C00832F8A50805D0E94EA0A0F7E351769F453
:100C6C0080E2B2D48FE6B0D48BE6AED48DE0ACD4B7
:100C7C00F1E0E4E05A950CD508950C942205086037
:100C8C009170F92F0E948D0AEEF7E92F9F2B09F432
:100C9C00F2E00E94A30B0E948D0AEEF7077F092E4B
:100CAC0030912701409128010E94C10D30932701FA
:100CBC0040932801089582E0E0D226F4442311F4F5
:100CCC0068940895E894089583E00E940A0916F444
:100CDC000E94A40D089583E00E940A0926F40E9444
:100CEC00A40D0E94BB0D08950E94FB0856F40E94AF
:100CFC00A60B03C00E94FB0826F430932A010E9425
:100D0C00BB0D089583E00E940A090EF00895442358
:100D1C0071F580912701909128018F3F08F027C031
:100D2C008F939F93E82FF92FFE5F008000922A018A
:100D3C0001968093270190932801332389F03F93E8
:100D4C008F939F930E94BB0D9F918F913F91019622
:100D5C00803031F080932701909328013A9569F700
:100D6C009F91909328019F9190932701089564CEB1
:100D7C000E94FB080EF00895309331010E94FE0C86
:100D8C0008950E94FB080EF0089530953695309327
:100D9C0033010E94FE0C08950E94FB080EF008958A
:100DAC00309332010E94FE0C089583E00E940A09E0
:100DBC000EF00895393C08F03FCE309330013436B4
:100DCC0011F430E820C0393B10F096E015C03639EC
:100DDC0010F095E011C0383710F094E00DC03535A7
:100DEC0010F093E009C0323310F092E005C03F30B0
:100DFC0010F091E001C09927532F56955695350F59
:100E0C00390F08F43FEF30932F01089583E00E94CF
:100E1C000A090EF00895442329F43A3518F4309356
:100E2C003A0110C009CE83E00E940A090EF0089521
:100E3C004423C1F73A35B0F73130A1F330933B017D
:100E4C00332309F031E030933E01332730933C01DA
:100E5C00089583E00E940A090EF0089530933D0135
:100E6C0030933E0108953F934F93EF93FF938091FE
:100E7C003D0180933E0180913C019927442730919C
:100E8C003A01380F3A3508F033270E94640CFF9171
:100E9C00EF914F913F9180913C01839590913B0153
:100EAC00891709F4882780933C01089583E00E94F8
:100EBC000A090EF00895442309F021C0313808F0D6
:100ECC0030E883E70E94EA0A90912601809125017F
:100EDC000E94920986E70E94EA0AF5E0E09125015A
:100EEC00EA9581910E948109E03031F03A9521F028
:100EFC008CE20E94EA0AF5CF0E94E90A08959CCD83
:100F0C000F921F9283E40E94EA0A88E40E94EA0A84
:100F1C008DE30E94EA0A80912501682F90912601A9
:100F2C000E94920980E20E94EA0AF0912801E09165
:100F3C002701FE5F508186E40E94EA0A89E60E943E
:100F4C00EA0A8EE60E94EA0A8DE30E94EA0A852FDD
:100F5C000E94810980E20E94EA0AF0912801E09146
:100F6C0027016E2F51915F9384E50E94EA0A88E570
:100F7C000E94EA0A8DE30E94EA0A852F0E948109E9
:100F8C0080E20E94EA0A82E50E94EA0A8DE30E944E
:100F9C00EA0A5F91852F90912F01903841F0899F3B
:100FAC00812D803810F08FEF02C0000C881F0E943A
:100FBC00810980E20E94EA0A6F3F91F187E40E9466
:100FCC00EA0A8DE30E94EA0A819190912F019038F0
:100FDC0041F0899F812D803810F08FEF02C0000CFA
:100FEC00881F0E94810980E20E94EA0A6E3FC1F0CC
:100FFC0082E40E94EA0A8DE30E94EA0A80819091C1
:10100C002F01903841F0899F812D803810F08FEF9F
:10101C0002C0000C881F0E94810980E20E94EA0A2B
:10102C000F938DE40E94EA0A86E40E94EA0A8DE39B
:10103C000E94EA0A0F7B809130010E94F40985E23C
:10104C000E94EA0A80E20E94EA0A83E40E94EA0A09
:10105C0083E50E94EA0A8DE30E94EA0A80913A0134
:10106C000E94F4098FE20E94EA0A80913B010E94DF
:10107C00F4098FE20E94EA0A80913D018F770E9469
:10108C00F40980E20E94EA0A84E50E94EA0A8DE3F0
:10109C000E94EA0A80912B010E94F4098EE20E94C0
:1010AC00EA0A80912C010E94F4090F918DE00E94B4
:1010BC00EA0A1F900F900895992790932B01909313
:1010CC002C0183E0A1D00EF0B7CC423008F0B4CCA8
:1010DC005F9355279927442311F099E156E0332368
:1010EC0061F03A3018F03A509395FBCF350F3A3007
:1010FC0010F03A5093955F9102C0352F5F9190326A
:10110C0010F09FE139E090932B013A3008F039E070
:10111C0030932C0100244427990F892F990F990F94
:10112C00890F041E890F041E890F041E890F041ECB
:10113C00890F041E890F041E880F001C330F432FC8
:10114C00330F330F340F4427830F041E00922D01ED
:10115C0080932E0108959EE78CEE0E942C0B9FE746
:10116C0080E20E942C0B9FE782EE0E942C0BF1E098
:10117C00E8E00E94430B902D0E94430B802D892B9D
:10118C0011F0802D02C091E483E20F930062F19A7A
:10119C003BD2F198892F38D29FE788EE0E942C0B16
:1011AC00F1E0EAE00E94430B802D0E94430B502D8E
:1011BC000E94430B002011F0952F02C087E390E0B2
:1011CC00F79902C092E886E3582F892FF19A1CD226
:1011DC00F198852F19D28DE0F7D19FE780E80E9416
:1011EC002C0B0F9108950C94220506FF04C082E08D
:1011FC0044D03EF403C083E007D01EF4442311F422
:10120C00689408950C94220582D1F6F7332744276D
:10121C008F9302C07CD1F6F79D3039F19A3029F1C9
:10122C00903278F0B9F39C32A9F39E3299F3903353
:10123C00E0F09734D0F4913420F49A33B0F452D0D7
:10124C0016F00C942205330F441F532F642F330FC9
:10125C00441F330F441F350F461F6627390F461F97
:10126C008A95C1F668948F91089500619F918917B2
:10127C0011F4E8940895689408958F9333274427C4
:10128C0046D1F6F79D3089F3973F11F49DE0EDCFF1
:10129C009032E8F0A9F3903340F3973430F791345F
:1012AC0010F49A3310F718D016F00C942205330F63
:1012BC00441F330F441F330F441F330F441F662743
:1012CC00390F461F8A95E1F668948F9108950C9416
:1012DC002205913470F002C0913420F0973448F418
:1012EC00975305C0903328F090539A3010F46894BB
:1012FC000895E89408959F93992706FF0AC08F9349
:10130C0084E2F79961D10000F79BF9D98F9166D0EF
:10131C0001C064D09F9108950F930F7D5F936F93DD
:10132C003F92582F992369F19732B0F011F4503154
:10133C0098F087E2382E60E18827931540F011F47D
:10134C00561728F083950062561B9309F6CF8063DD
:10135C00F7993AD1F79BD3D983E0382E68EE8827DA
:10136C00931540F011F4561728F083950062561B24
:10137C009309F6CF806305FF04C0F79925D1F79B3D
:10138C00BED98827332464E6992311F4561728F024
:10139C0083950062561B9309F7CF806305FF04C049
:1013AC00F79912D1F79BABD988276AE0561720F032
:1013BC0083950062561BFACF806305FF04C0F79932
:1013CC0003D1F79B9CD9852F8063F799FDD0F79BB0
:1013DC0096D93F906F915F910F9108950F9306FFEF
:1013EC001BC09F93982F82958F7005FD41F0805DF7
:1013FC008A3308F0895FF799E7D0F79B80D9892F5A
:10140C008F70805D8A3308F0895FF799DDD0F79B88
:10141C0076D99F910F9108959F935F93982F88276A
:10142C00943660F054E680E38395951B9436E0F790
:10143C009F93F799C9D0F79B62D99F91882311F498
:10144C009A3068F05AE080E39A3018F08395951B37
:10145C00FBCF9F93F799B8D0F79B51D99F91892FC8
:10146C00805DF799B1D0F79B4AD95F919F910F910D
:10147C000895A89501FF47C00D7F992790933701D8
:10148C00F09918C012FD0E940B0E02FF13C00B7FC7
:10149C0090913B01992371F080913D01882351F08B
:1014AC0080913E01882331F08A9580933E0111F49E
:1014BC000E94390700FF1DC00E7F14FD06C00000FE
:1014CC00F09B03C0F0982E9A5D9ACBD080911B01B3
:1014DC00891779F02E985D98F8940E945D0B81E045
:1014EC008EBF8CEF8DBF7894A8950E94650B0C94E1
:1014FC005B0380911501882331F08A958093150147
:10150C0011F42E9A5D9A13FD0E944C0E08958F9340
:10151C00EF93FF93AEDF04FF04C0909138010F7E70
:10152C003CC0E894F82DE92D972D9E1721F4962DAB
:10153C009F1709F444C09191F53011F4F2E0E0E00A
:10154C008F2E9E2E5F936F93572D662D681430F05F
:10155C0009F005C0791410F0E1F001C06D5F591964
:10156C006809623010F0503BA0F410FF12C01E7FCF
:10157C00F8940000F2E0F093E900F091E800FB7FB2
:10158C00F093E8000000F091E800FF77F093E8009A
:10159C0078946F915F9190933801F79B07C003FD8E
:1015AC0005C09B3718F4913608F090520F7E689462
:1015BC00F09905C0E9E1E09315012E985D98FF9133
:1015CC00EF918F9108958DE08F93F894000081E056
:1015DC008093E900A8958091E80080FFFBCF8E7B7B
:1015EC008093E8008F918F938093F1008091E800B5
:1015FC008E7F8093E80000008091E8008F778093C5
:10160C00E80078948F9108958F9305FD02C080E2D5
:10161C00DBDF8F918F9382958F70805D8A3308F01A
:10162C00895FF19908C0F29B02C0803329F08033A6
:10163C0011F4F19B80E2C8DF8F918F938F70805DE6
:10164C008A3308F0895FC0DF8F910895FF93EF9381
:10165C00FC018591882311F0B7DFFBCFEF91FF914F
:10166C0008954F9B05C09927F79AF498F39804C0F6
:10167C009FEFF79AF49AF39A089503D00094319659
:10168C000895F2BDE1BD002403940FBA00B408958F
:10169C00509502D031960895A895F894F2BDE1BD0D
:1016AC0050BDFA9AF99AF999FECF789408959F93C0
:1016BC009AEFA8950AD09A95E1F79F910895F7DFD4
:1016CC00F6DFF5DFF4DFF3DF08959F9398EC9923B1
:1016DC0049F09F939F919F939F9100000000000001
:1016EC009A95F5CF9F910895002491E09093D7009F
:1016FC0090EB9093D80000009F7D9093D800000051
:10170C0090629093D80090E199BD926099BD99B583
:10171C0090FFFDCF9091D8009F7D9093D800992792
:10172C009093E00098E09093E20092E0692E892E6D
:10173C0090E0792E992E78940895FB5F3197089557
:10174C00E0912501F0912601FF2361F43196E0939D
:10175C002501F09326010E94A30BF0932801E0933E
:10176C00270108950C942205F0912801E09127019E
:10177C005081FE5F0080902D9F3F49F003940082C2
:10178C0000922A01F250951719F4008201C0F25010
:10179C000895F0912801E09127015081FE5F0080AF
:1017AC00902D9923A1F30A94EACF82E00E940A09B2
:1017BC00C6F53A3510F00C94220513FFFECFAF930B
:1017CC00BF93EF93FF933F93F4E2F30FEE27A0E068
:1017DC00B7E09BE5909337010E94023FE0E89BE560
:1017EC00909337010E94023F9927909337013F91C4
:1017FC00332399F4F1E0E0E050912D010E944E0B5F
:10180C0050912E010E944E0B5FEF06FD55270E9452
:10181C00520B3196522F0E944E0BFF91EF91BF91BC
:10182C00AF91089582E00E940A09DEF73A3510F074
:10183C000C9422053323B1F4F1E0E0E00E94430B59
:10184C0000922E010E94430B00922D010E94470B27
:10185C000F7B01FE006431960E94430B902D907F0C
:10186C002F70292BAF93BF93EF93FF93F4E2F30FF9
:10187C00EE27A0E0B7E0A895059000940D92A0305B
:10188C00D9F7F5E0E0E0B7E0A0E0A8950C90508126
:10189C00501559F080912E0190912D01992321F42E
:1018AC00882311F4008201C080D131961196F63054
:1018BC0061F7FF91EF91BF91AF9108953A3510F018
:1018CC000C942205AF93BF93EF93FF93F4E2F30FC5
:1018DC00EE27A0E0B7E0A895059000940D92A138F2
:1018EC00D9F7F5E0E0E0B7E0A0E0A8950C905081C6
:1018FC00501559F080912E0190912D01992321F4CE
:10190C00882311F4008201C050D131961196E13830
:10191C0061F7FF91EF91BF91AF9108959FE788ED2B
:10192C0095DE0E948D0AEEF79F7D943411F00C9495
:10193C0022058DE049DEF894F5E0E0E0B7E0A0E0A8
:10194C0099279193F49905C09D93F630D1F778942B
:10195C000895F730B1F7789408959FE788ED76DE17
:10196C000E948D0AEEF79C3711F00C942205F89426
:10197C00F1E0E4E055278CDEA2DEA1DEA0DE8DE0F6
:10198C000E94EA0AF894F5E0E0E099279193FB3085
:10199C00E9F70F7B1F7B992790932A0190932B01DA
:1019AC0090932C0190932D0190932E0190932601EE
:1019BC0082E380933A0190933B019093390184E147
:1019CC0080933D01939590932501909333019FEF64
:1019DC009093320190E890932F0194E6909330010C
:1019EC0095E09093280190E09093270178940895C6
:1019FC00309131013B3238F4330F5FEF531B330F0F
:101A0C00632F882742C0353580F43B52432F4695CF
:101A1C00469546956BEA330F630F330F3395339529
:101A2C005CEA531B541B882730C0303840F43555C2
:101A3C00330F6FEF631B330F832F552726C03A3AB2
:101A4C0080F43058432F4695469546958BEA330FD4
:101A5C00830F330F339533956CEA631B641B552747
:101A6C0014C0353D40F43A5A330F8FEF831B330FBC
:101A7C00532F66270AC0355D5BEA330F530F330FC4
:101A8C00339533958AEA831B66271F929091330115
:101A9C009F779923C1F09F3709F490E84FEF451BCE
:101AAC00499F412D000C441F540F4FEF461B499F7B
:101ABC00412D000C441F640F4FEF481B499F412DD3
:101ACC00000C441F840F909132019F3F69F0969552
:101ADC00599F512D000C551F699F612D000C661FDD
:101AEC00899F812D000C881F1F9060933501809376
:101AFC003601309125014091260150932A010E9414
:101B0C00BB0D0090350100922A010E94A60B0E9489
:101B1C00BB0D0090360100922A010E94A60B0E9478
:101B2C00BB0D3093250140932601E32FF42F0E9427
:101B3C00A30BF0932801E09327010895442329F087
:101B4C00423088F4332379F402C0332361F03093AC
:101B5C00250140932601E32FF42FEFDDF0932801AC
:101B6C00E093270108950C942205F0912801E0914F
:101B7C00270100902A0100922A01F0932801E0939A
:101B8C0027015081501509F40EC0FE5F0082F250FF
:101B9C0080912E0190912D01992321F4882311F429
:101BAC00008201C002D078940895501908F4519520
:101BBC00002480912E0190912D010AD0FD5F90831D
:101BCC00F39580838827F3958083F55014600895EE
:101BDC004F923324441861E1001C551F6A9551F44F
:101BEC009695879583199409802D952F08F4019665
:101BFC004F900895331C441C381A490A20F4380EAF
:101C0C00491E8894E9CF0894E7CF5F936F933F9276
:101C1C00F5E0E0E01B7F8081FE5F9081891711F475
:101C2C00F2501DC0F3955081F3956081F39530808F
:101C3C00360E08F453953082891740F4850F20F046
:101C4C00981710F0146009C0892F07C0851B20F06D
:101C5C00891710F0146001C0892FF55080833196DC
:101C6C00E03009F0D8CF3F906F915F910895599A69
:101C7C0093E09093CC009091C8009D7F9093C80006
:101C8C0099279093C9009EE09093CA000E946B0B19
:101C9C00F8949091C900977B9093C9005B98539AE4
:101CAC0078940E946B0B5B9A14D01FD0F89495E03B
:101CBC00F92EEE249091C90098649093C90099274D
:101CCC009093CE00177F789408959F9392E00C9494
:101CDC006D0B9F9390E10C946D0B9F9390EB0C9478
:101CEC006D0B9F9390E00C946D0B9F9394E00C9470
:101CFC006D0B12011001020000080E010000000122
:101D0C0009024300020100803109040000010202B3
:101D1C00000005240010010524010300042402071F
:101D2C000524060001070583031000400904010087
:101D3C00020A0000000705810240000107050202AB
:101D4C004000010009024300020100803109040037
:101D5C00000102020000052400100105240103000B
:101D6C000424020705240600010705830310004024
:101D7C0009040100020A000000070581024000402E
:101D8C00070502024000000A120355006E002000F5
:101D9C004B006E006F0077006E001C035500530063
:101DAC0042002D00530069006D0070006C0065004E
:101DBC0044006D00780000C2010000000800000023
:101DCC0012010002010000080E01000100010902CD
:101DDC0065000201008031090400000001010000CF
:101DEC000924010001090001010904010002010399
:101DFC000000072401000141000624020101000635
:101E0C002402020200092403010301020100092437
:101E1C0003020401010100090581024000000000D9
:101E2C0005250101030905020240000000000525FB
:041E3C00010101009F
:0223FE000000DD
:10780000FFFFFF00FFFFFFFFFFFFFFFFFFFFFFFF87
:06781000FFFFFF5060FFC6
:10790000FFFFFF4040FFFFFFFFFFFFFFFFFFFFFF05
:06791000FFFFFF00FFFF76
:107A0000FFFFFFFF00FFFFFFFFFFFFFFFFFFFFFF85
:067A1000FFFF4040FFFFF4
:107B0000FFFFFFFF5060FFFFFFFFFFFFFFFFFFFFD3
:067B1000FFFF00FFFFFF74
:107C0000FFFFFFFFFF00FFFFFFFFFFFFFFFFFFFF83
:067C1000FFFF60FF60FFB2
:107D0000FFFFFF60FF60FFFFFFFFFFFFFFFFFFFFC1
:067D1000FFFFFFFF00FF72
:107E00000C9408035F938F939F93EF93FF93F43247
:107E100020F4FE3710F00C942205F999FECF9091D2
:107E200037019B3511F00C94220599279093370167
:107E3000F89493E00E94423F91E10E94423F80E427
:107E40000D901D900094109491E00E94423F329654
:107E50008A95B1F7FF91EF91EF93FF9395E00E9420
:107E6000423F91E10E94423F87B786FF04C091E103
:107E70000E94423FF9CF7894FF91EF919F918F91AB
:107E80005F91089557B750FDFDCF97BFE8950895CE
:107E90000F7B0895006408950E94FB087EF4F09122
:107EA0002801E0912701FE5F9081930F08F49FEF76
:107EB000092E90932A01F2500E94C10D08950E944C
:107EC000FB08E6F7F0912801E0912701FE5F908121
:107ED000931B70F79927ECCFE0E0F5E0A0E0B7E066
:107EE00091919D93F630E1F71B7F08950D73696DB5
:107EF000706C65205553422F444D5820496E74656F
:107F0000726661636520666F722041726475696E86
:107F10006F204D6963726F202876312E313429002D
:107F200020286329323031352D323120572E5363CA
:107F300068656D6D6572740D00004A756D706572CF
:107F4000204F46463A41534349495F636D64536548
:107F500074202B204D696E69444D582C32353663A0
:107F6000680D4A756D706572204F4E3A4D4944490F
:107F70005F636D645365742C32353663680D0000A1
:107F80004A756D706572204F46463A4153434949E0
:107F90005F636D64536574202B204D696E69444D99
:107FA000582C32353663680D4A756D706572204FF6
:107FB0004E3A6F6E6C79204D696E69444D5820625F
:107FC00075742035313263680D004D494449206392
:107FD0006828312D31362900205265706561742082
:0E7FE00000005649443D0000205049443D0039
:00000001FF
